:100000000C9468050C94B0050C94B0050C94B005E4
:100010000C94B0050C94B0050C94B0050C94B0058C
:100020000C94B0050C94B0050C94B0050C949F1D75
:100030000C94B0050C94761D0C94B0050C94B0058E
:100040000C94B0050C94B0050C94B0050C94501DA4
:100050000C94B0050C94B0050C94B0050C94672278
:100060000C94B0050C94B0050C94B0050C94B0053C
:100070000C94B0050631FF0974A10109751500261D
:10008000FF009520750881020976150026FF00956E
:100090002075089102C005010902A1010901A10012
:1000A0008501050919012908150025019508750123
:1000B00081020501093009311581257F95027508F6
:1000C000810609381581257F950175088106050C83
:1000D0000A38021581257F950175088106C0C00583
:1000E000010980A10185021601002637001A81004E
:1000F0002AB700751095018100C0050C0901A10106
:100100008503160100269C021A01002A9C02751024
:1001100095018100C005010906A101050719E02923
:10012000E715002501950875018102950175088183
:1001300001050819012905950575019102950175BB
:100140000391010507190029FF150026FF009506F8
:1001500075088100C020002530325800646F6E653C
:100160002E0A00626F6F746D61676963207363614B
:100170006E3A202E2E2E200025583A253038622542
:10018000730A000A202030313233343536370A0002
:100190004C45443A20253032580A000A4C6F6F70A3
:1001A0002073746172742E0A000A55534220636FE3
:1001B0006E666967757265642E0A000A544D4B3A83
:1001C0003131333162352F4C5546413A643661370F
:1001D00064660A0009025400030100A03209040009
:1001E0000001030101000921110100012240000763
:1001F00005810308000A0904010001030102000946
:100200002111010001227F00070582030800010976
:100210000402000103000000092111010001222253
:1002200000070583032000011201100100000008EF
:10023000EDFE21500100010200013A0353004F007E
:100240004E00590020004E0045005700530020008A
:100250006B006500790062006F006100720064004D
:10026000200063006F006E0076006500720074006D
:100270006500720000000E0374002E006D002E0059
:100280006B002E0000000403090473797374656D1C
:100290003A20253034580A00636F6E73756D6572AD
:1002A0003A20253034580A003F004D3E2000433E9E
:1002B00020000A00257500363A20776865656C5F76
:1002C00074696D655F746F5F6D61783A20000A0034
:1002D000257500353A20776865656C5F6D61785FDC
:1002E00073706565643A20000A00257500343A2071
:1002F00074696D655F746F5F6D61783A20000A0004
:10030000257500333A206D61785F73706565643AD6
:1003100020000A00257500323A20696E74657276F5
:10032000616C286D73293A20000A00257500313A66
:100330002064656C6179282A31306D73293A200078
:100340000A092D2056616C756573202D0A004D3EFB
:10035000004D25643E20003F00736574206465668F
:1003600061756C740A00433E20000A002530325843
:1003700020006B6579626F6172643A2000803A3BBD
:100380003C3D3E3F40414243291E1F202122232461
:100390002526272D2E742A2B141A0815171C180C25
:1003A00012132F304C78041607090A0B0D0E0F3369
:1003B000343228791D1B0619051110363738757D22
:1003C0007A39772C7665007C5F6061565C5D5E579C
:1003D000595A5B666252635850514F8080808080CA
:1003E000805554678044454A494D4B4E80808080FB
:1003F00080808080808080038080808080290A00C7
:100400002575002F002575005D280025640020005B
:10041000256400200025640020002564007C002560
:10042000303258006D6F7573656B6579205B62744F
:100430006E7C782079207620685D287265702F6147
:10044000636C293A205B006D6F7573653A205B25FC
:100450003032587C25642025642025642025645D85
:100460000A000A002575002E6E6B726F3A20000A92
:10047000002575002E737761705F6261636B736C2A
:100480006173685F6261636B73706163653A2000DA
:100490000A002575002E737761705F67726176655B
:1004A0005F6573633A20000A002575002E6E6F5F4A
:1004B0006775693A20000A002575002E7377617010
:1004C0005F72616C745F726775693A20000A00257B
:1004D00075002E737761705F6C616C745F6C67750B
:1004E000693A20000A002575002E636170736C6FF5
:1004F000636B5F746F5F636F6E74726F6C3A200032
:100500000A002575002E737761705F636F6E7472D9
:100510006F6C5F636170736C6F636B3A20000A00ED
:1005200025303258006B65796D61705F636F6E6660
:1005300069672E7261773A20000A002575002E6DDA
:100540006F7573653A20000A002575002E6B65797A
:10055000626F6172643A20000A002575002E6D6199
:10056000747269783A20000A002575002E656E6164
:10057000626C653A20000A002530325800646562DA
:1005800075675F636F6E6669672E7261773A2000E8
:100590000A0025750064656661756C745F6C61792D
:1005A00065723A20000A092D204D61676963202D8C
:1005B0000A643A0964656275670A783A0964656293
:1005C0007567206D61747269780A6B3A09646562B7
:1005D0007567206B6579626F6172640A6D3A0964B0
:1005E00065627567206D6F7573650A763A09766581
:1005F0007273696F6E0A733A097374617475730A62
:10060000633A09636F6E736F6C65206D6F64650A82
:10061000302D343A096C61796572302D34284631B9
:10062000302D4634290A506175733A09626F6F7430
:100630006C6F616465720A653A09656570726F6D09
:100640000A000A092D20436F6E736F6C65202D0A16
:100650004553432F713A09717569740A6D3A096DF2
:100660006F7573656B65790A003F0074696D65721B
:100670005F72656164333228293A202530346C5822
:100680000A006B6579626F6172645F69646C653AD8
:100690002025580A006B6579626F6172645F707221
:1006A0006F746F636F6C3A2025580A00686F73741B
:1006B0005F6B6579626F6172645F6C656473282932
:1006C0003A2025580A000A092D2053746174757365
:1006D000202D0A004743433A20372E332E30204145
:1006E00056522D4C4942433A20322E302E30204172
:1006F00056525F415243483A2061767233350A00C0
:100700004F5054494F4E533A204C55464120424F8A
:100710004F544D41474943204D4F5553454B455943
:100720002045585452414B455920434F4E534F4C4E
:100730004520434F4D4D414E44204B45594D41506E
:100740005F53454354494F4E20343039360A0042F6
:1007500055494C443A203131333162352028323208
:100760003A30383A3133204E6F7620203220323002
:100770003233290A005649443A20307846454544E8
:1007800028742E6D2E6B2E29205049443A20307843
:100790003530323128534F4E59204E455753206B38
:1007A0006579626F61726420636F6E7665727465DD
:1007B0007229205645523A203078303030310A00C4
:1007C000444553433A20636F6E76657274732053C9
:1007D0004F4E59204E4557532070726F746F636FA0
:1007E0006C20696E746F205553420A000A092D204F
:1007F00056657273696F6E202D0A000A6D6F7573EE
:10080000653A206F66660A000A6D6F7573653A2057
:100810006F6E0A000A6B6579626F6172643A206FCD
:1008200066660A000A6B6579626F6172643A206FCE
:100830006E0A000A6D61747269783A206F66660A02
:10084000000A6D61747269783A206F6E0A000A645A
:10085000656275673A206F6E0A000A6465627567A3
:100860003A206F66660A000A0A626F6F746C6F61E5
:100870006465722E2E2E2000433E20006565636F56
:100880006E6669673A0A006D6B5F776865656C5FD5
:1008900074696D655F746F5F6D6178203D202564BC
:1008A0000A006D6B5F776865656C5F6D61785F737B
:1008B00070656564203D2025640A006D6B5F746976
:1008C0006D655F746F5F6D6178203D2025640A005F
:1008D0006D6B5F6D61785F7370656564203D202589
:1008E000640A006D6B5F696E74657276616C203DA1
:1008F0002025640A006D6B5F64656C6179203D2082
:1009000025640A006D6B5F776865656C5F74696D5F
:10091000655F746F5F6D6178203D2025640A006D0E
:100920006B5F776865656C5F6D61785F7370656537
:1009300064203D2025640A006D6B5F74696D655FFE
:10094000746F5F6D6178203D2025640A006D6B5FD8
:100950006D61785F7370656564203D2025640A00D1
:100960006D6B5F696E74657276616C203D202564E5
:100970000A006D6B5F64656C6179203D2025640A17
:100980000077686572652064656C74613A206375F0
:1009900072736F723D25642C20776865656C3D2508
:1009A000640A53656520687474703A2F2F656E2E43
:1009B00077696B6970656469612E6F72672F7769FB
:1009C0006B692F4D6F7573655F6B6579730A000AEC
:1009D000092D204D6F7573656B6579202D0A455380
:1009E000432F713A09717569740A313A0964656C6B
:1009F0006179282A31306D73290A323A09696E7497
:100A0000657276616C286D73290A333A096D6178D5
:100A10005F73706565640A343A0974696D655F7463
:100A20006F5F6D61780A353A09776865656C5F6D4F
:100A300061785F73706565640A363A097768656541
:100A40006C5F74696D655F746F5F6D61780A0A70C1
:100A50003A097072696E742076616C7565730A6408
:100A60003A097365742064656661756C74730A7500
:100A7000703A092B310A646F776E3A092D310A708A
:100A80006775703A092B31300A7067646F776E3A78
:100A9000092D31300A0A7370656564203D20646554
:100AA0006C7461202A206D61785F737065656420C5
:100AB0002A2028726570656174202F2074696D6525
:100AC0005F746F5F6D6178290A004C25640A00002D
:100AD00011241FBECFEFD4E0DEBFCDBF04B603FEAE
:100AE00028C08091DD029091DE02A091DF02B091DA
:100AF000E0028730904BA740B04BD9F41092DD0252
:100B00001092DE021092DF021092E00214BE0FB6C5
:100B1000F894A8958091600088618093600010929D
:100B200060000FBE1092010810920008E0E0F8E3A8
:100B3000099511E0A0E0B1E0ECE7F8E402C005900F
:100B40000D92A233B107D9F722E0A2E3B1E001C0D0
:100B50001D92AD3DB207E1F70E946E1E0C943C243D
:100B60000C940000FF93EF93E0913201F091330178
:100B7000309709F00995EF91FF910895FC01859157
:100B8000803011F0EFDFFBCF0895FF27E0E230E285
:100B900047FF0CC0419597FF09C0EDE26095709545
:100BA00080959095611D711D811D911D27FF02C0CB
:100BB000219530E350E2AA27660F771F881F991FFF
:100BC000AA1FA41710F0A41B63955A95A9F7AA3081
:100BD00008F0A95FA05DAF93F395611571058105DC
:100BE000910541F7ED3211F4EF93F395F21718F4F4
:100BF0003F93F395FBCF8F91B5DFFA95E1F7089519
:100C0000E991F9918591803021F0853219F0AADFC0
:100C1000F9CF089520E0E89455915532C1F350334F
:100C200011F4689455915A3348F4505390F3220FBD
:100C3000022E220F220F200D250FF4CF0EF4219546
:100C400089919991533619F3533729F1533559F155
:100C5000BC0188279927E8945C3621F48991999101
:100C600068945591543639F446EF7EF077FF0DC005
:100C70008FEF9FEF0AC055374AE039F0583540E111
:100C800021F0523642E009F00895FF93EF937DDFA3
:100C9000EF91FF91B7CFFF93EF93FC0181918030EB
:100CA000B9F360DFFBCFFF93EF9368DFF1CFDF9302
:100CB000CF93CDB7DEB72596A3DFCF91DF9108950F
:100CC000803FC1F48091CF0287FD1092CF028091C6
:100CD000CE0281110EC08091CF0281110AC0809195
:100CE000D002811106C08091D102811102C0109200
:100CF000C8020895813F29F48091CF0218162CF381
:100D0000E6CF9091CE02823F29F497FFE0CF109278
:100D1000CE02DDCF833F19F41916CCF3D8CF893F2B
:100D200039F48091D002181694F61092D002CFCFE9
:100D30008A3F29F48091D00287FFC9CFF6CF8B3F3D
:100D400039F48091D10287FFC2CF1092D102BFCF78
:100D50008C3F29F48091D1021816BCF3B8CF843FA0
:100D600031F48091CD028E7F8093CD02B0CF853F4C
:100D700021F48091CD028D7FF7CF863F21F48091C1
:100D8000CD028B7FF1CF873F21F48091CD02877F09
:100D9000EBCF883F21F48091CD028F7EE5CF8D3F50
:100DA00031F48091C7028E7F8093C70290CF8E3F2F
:100DB00021F48091C7028D7FF7CF8F3F09F087CF55
:100DC0008091C7028B7FF0CF8091C70280FF0CC05B
:100DD0006091130170E0759567957595679561153C
:100DE000710559F1862F089581FF06C060911301A6
:100DF00070E075956795F3CF6091130170E082FD07
:100E00000CC06091C8026623A9F020911201809164
:100E1000130190E0621730F0BC0160387105F8F200
:100E20008FE7089570E00E94FD23622F70E00E941A
:100E30000E24F3CF61E070E0D5CF81E0089580917A
:100E4000C70280FF11C08091150190E065E070E05D
:100E50000E94FD23959587959595879580389105F6
:100E6000B0F50097B1F1089581FF0AC08091150196
:100E700090E065E070E00E94FD2395958795EECFA8
:100E800082FF08C08091150190E065E070E00E944B
:100E9000FD23E4CF3091C8023323B1F02091140137
:100EA0008091150190E065E070E00E94FD23BC0197
:100EB0003217A0F6832F90E00E94FD23622F70E08E
:100EC0000E940E24CB01CACF85E090E008958FE701
:100ED000089581E00895803F31F40E941F078195B5
:100EE0008093CF020895813F19F40E941F07F8CF25
:100EF000823F31F40E941F0781958093CE020895AE
:100F0000833F19F40E941F07F8CF893F29F40E94FC
:100F1000E4068093D00208958A3F21F40E94E406FB
:100F20008195F7CF8B3F31F40E94E4068195809341
:100F3000D10208958C3F19F40E94E406F8CF843F53
:100F400031F48091CD0281608093CD020895853F78
:100F500021F48091CD028260F7CF863F21F4809109
:100F6000CD028460F1CF873F21F48091CD0288606B
:100F7000EBCF883F21F48091CD028061E5CF8D3F9A
:100F800031F48091C70281608093C70208958E3F3B
:100F900021F48091C7028260F7CF8F3FB9F780912B
:100FA000C7028460F1CFE72FF0E093E0EE0FFF1F60
:100FB0009A95E1F7E60FF11DE358FC4F6491E62F97
:100FC000E295E77090E023E0880F991F2A95E1F7FA
:100FD0008E0F911D34E0880F991F3A95E1F7E62FA7
:100FE000EF70E80FF92FF11DEE0FFF1FE050F849E9
:100FF000859194910895AF92BF92CF92DF92EF9234
:10100000FF921F93CF93DF935C0187EBC82E82E0A2
:10101000D82E10E0F601E1906F01D0E0C0E0F12C95
:10102000C7010C2E02C0959587950A94E2F780FFC0
:101030001DC06C2F712F80E00E94D3078A159B057D
:1010400051F0292F207E392F307C11F0203A71F495
:101050008A151B0459F481E0DF91CF911F91FF9015
:10106000EF90DF90CF90BF90AF9008952196C83059
:10107000D105B1F61F5F103169F680E0EDCFCF9357
:10108000DF93EC018CE290E00E94FB07882329F0BB
:10109000CE01DF91CF910C94FB0780E0DF91CF91DF
:1010A00008952FB7F8948091D2029091D302A09125
:1010B000D402B091D5022FBF08954F925F926F92E4
:1010C0007F929F92AF92BF92CF92DF92EF92FF9268
:1010D0000F931F93CF93DF9300D000D01F92CDB713
:1010E000DEB76B837C838D837A018C819D81892B14
:1010F00049F08FEFF81204C081E09FEF491719F013
:1011000080E001C081E080FD6AC00F2D10E0CE2C90
:10111000D12C8B81882309F456C040902F02509027
:10112000300260903102709032028091D902909129
:10113000DA02A091DB02B091DC02482A592A6A2A1D
:101140007B2A2FE1A22EB12C9A2CD301C2010A2CAA
:1011500004C0B695A795979587950A94D2F780FD18
:101160002BC081E0A81AB10878F7912CF80193E020
:10117000EE0FFF1F9A95E1F7ED5CFD4FEC0DFD1DA5
:101180009082E982FA8269817A81892D0F900F908D
:101190000F900F900F90DF91CF911F910F91FF90C3
:1011A000EF90DF90CF90BF90AF909F907F906F9027
:1011B0005F904F900C94D307B7018A2D0E94D307FC
:1011C000019779F2D3CFF80183E0EE0FFF1F8A95E4
:1011D000E1F7ED5CFD4FEC0DFD1D9080D2CF90E06E
:1011E00080E00F900F900F900F900F90DF91CF91B4
:1011F0001F910F91FF90EF90DF90CF90BF90AF9035
:101200009F907F906F905F904F90089541E050E0E5
:1012100060E070E004C0440F551F661F771F8A9579
:10122000D2F7409550956095709580912F029091DE
:101230003002A0913102B091320284239523A6237B
:10124000B72380932F0290933002A0933102B09382
:101250003202089541E050E060E070E004C0440FC5
:10126000551F661F771F8A95D2F780912F029091A4
:101270003002A0913102B0913202842B952BA62B23
:10128000B72B80932F0290933002A0933102B0933A
:101290003202089580912E029091FD01981301C0B1
:1012A00008958F5F8770FACF1F93CF93DF9300D09D
:1012B00000D01F92CDB7DEB7942F4983252F5A83D4
:1012C0006B837C838D834C815D8181E0452B31F084
:1012D0002F3F19F481E09F3F09F080E0182F117033
:1012E00080FD2CC049815A816B817C818D810E9457
:1012F0005D08292F22952F702C3078F42A30A8F41D
:1013000022502230C8F0812F0F900F900F900F9035
:101310000F90DF91CF911F9108952C3011F02F3055
:1013200091F793FB112710F9EECF803C28F0803E17
:1013300050F3815F833038F311E0E5CF10E0E3CF65
:10134000E091C902F091CA02309721F00190F0813A
:10135000E02D099480E008951092E2001092E100DF
:10136000E0EEF0E0808181608083E8EDF0E0808154
:101370008F77808319BCE3E6F0E080818160808311
:101380001092DB0108950E94AC09F89487E797E773
:10139000909301088093000887E090EBDC01809334
:1013A000DD029093DE02A093DF02B093E00288E1B9
:1013B0009CE00FB6F894A895809360000FBE9093C0
:1013C0006000FFCFFC018091EF019091F001861742
:1013D0009707A0F06115710529F49091E8009E77B8
:1013E0009093E80090E06115710551F4911108C0E7
:1013F0008091E80082FF32C080E00895BC01F2CF06
:101400008091F1018823B1F18530B1F18091E8003C
:1014100083FD2EC08091E80082FDEACF8091E80034
:1014200080FFE1CF2091F20030E06115710519F0E5
:101430002830310558F091E02830310509F090E06E
:101440002091E8002E772093E800CDCF8191809302
:10145000F100615071092F5F3F4FE7CF8091F1019B
:10146000882341F0853041F08091E80083FFC0CFB0
:1014700081E0089582E0089583E008952091E400DA
:101480003091E50085E69091EC0090FF06C09091C8
:10149000E80090FF06C080E008959091E80092FD7A
:1014A000FACF9091F101992391F0953091F09091BC
:1014B000EB0095FD10C04091E4005091E500241729
:1014C000350709F381509A01F1F684E0089582E02E
:1014D000089583E0089581E008958091E90187FFF0
:1014E00013C08091E80082FF06C08091E8008B77EE
:1014F0008093E80004C08091F1018111F2CF08953A
:101500008091F1018823D9F38091E80080FFF8CF22
:101510008091E8008E77ECCF982F9093E900242FEC
:10152000762F50E0891731F07091EC002091ED009A
:101530005091F00021FD07C09F5F953071F78093B7
:10154000E90081E008953091EB003E7F3093EB009D
:101550003091ED003D7F3093ED003091EB00316034
:101560003093EB007093EC002093ED005093F0006B
:101570002091EE0027FDE0CF80E008950F931F93A8
:10158000CF93DF93CDB7DEB7AA970FB6F894DEBF3F
:101590000FBECDBF8091F101882309F44EC1109197
:1015A000E9001F708091EC0080FF39C080E8182BA3
:1015B0001092E9008091E80083FF3CC1E9EEF1E080
:1015C00081EF91E02091F10021938E179F07D1F7D1
:1015D0008091EA01833009F470C018F5813009F474
:1015E00047C0823009F4DAC08091E80083FF14C15B
:1015F0008091E9019091EA019A3008F00DC1E92F3C
:10160000F0E0EB5FF44F0C942224DF0B050C0C0C84
:10161000050C0C0C670C890C0C0C840D910D80E0F2
:10162000C6CF8A3009F4A9C08B3009F47DC0893057
:10163000D9F68091E9018132B9F68091ED0190915E
:10164000EE01892B89F68091E800877F8093E8007E
:101650008091E80082FF2CC08091F1008093DD0131
:101660008091E8008B778093E8000E946D0ABCCFE0
:101670008091E901813A09F0B7CF8091E800877F36
:101680008093E8008091ED019091EE01892B61F04B
:1016900060E090E080E070E00E94E2098091E80064
:1016A0008B778093E800A0CF68E08EED91E0F3CFD8
:1016B0008091F1018111CCCF97CF8091E901813ADE
:1016C00009F092CF8091ED019091EE01892BA1F468
:1016D0008091E800877F8093E8008091E80080FF98
:1016E000FCCF809111018093F1008091E8008E770A
:1016F0008093E8000E946D0A8091ED019091EE01C7
:10170000019709F071CF8091E800877F8093E8000E
:101710008091E80080FFFCCF809110018093F10060
:101720008091E8008E779FCF8091E901813209F0A6
:101730005BCF8091ED019091EE01892B59F480915E
:10174000E800877F8093E8000E946D0A8091EB019A
:10175000809311018091ED019091EE01019709F0C4
:1017600043CF8091E800877F8093E8000E946D0A54
:101770008091EB018093100137CF8091E901813294
:1017800009F032CF8091E800877F8093E8000E94C3
:101790006D0A8091EC018093D60226CF8091E901F9
:1017A000813A09F021CF8091E800877F8093E8009B
:1017B0008091E80080FFFCCF8091D602AFCF8038C7
:1017C00089F0823849F58091ED018F70853020F5E0
:1017D0008093E9008091EB0085FB882780F91092C7
:1017E000E90006C08091E6019091E70191118260C5
:1017F0009091E800977F9093E8008093F100109219
:10180000F1008091E8008E7731C0282F2D7F21F4E0
:101810008823F1F0823079F18091E80083FF0AC0DB
:101820008091E800877F8093E8008091EB008062E0
:101830008093EB001F701093E900AA960FB6F894FE
:10184000DEBF0FBECDBFDF91CF911F910F910895E5
:101850008091EB01813001F7933009F080E08093B3
:10186000E7011092E9008091E800877F8093E8000B
:101870000E946D0AD1CF8091EB018111F2CF80914E
:10188000ED018F702FEF280F243030F68093E900A0
:101890002091EB0020FFE5CF933031F48091EB00F5
:1018A00080628093EB00DDCF9091EB00906190938C
:1018B000EB0021E030E001C0220F8A95EAF7209387
:1018C000EA001092EA008091EB008860EACF811173
:1018D000A3CF0091EB010F778091E3008078802BFC
:1018E0008093E3008091E800877F8093E8000E9466
:1018F0006D0A8091E80080FFFCCF8091E300806852
:101900008093E30083E0011101C082E08093F10144
:1019100083CF8058823008F07FCF2091EB01309147
:10192000EC012C3D83E03807A1F583E08A838AE24D
:1019300089834FB7F894DE01139620E03EE051E230
:10194000E32FF0E050935700E49120FF03C0E295AD
:10195000EF703F5FEF708E2F90E0EA30C0F0C796D7
:101960008D939D932F5F243159F74FBF8091E800ED
:10197000877F8093E8006AE270E0CE0101960E94C2
:10198000E2098091E8008B778093E80045CFC0960C
:10199000E7CF8091ED019091EE01432F5527433021
:1019A000510509F44FC078F54130510509F445C09F
:1019B00084E590E0E4EDF1E04230510509F02CCFF0
:1019C0002091E800277F2093E8002091EF013091DB
:1019D000F0018217930708F49C0140E021153105BE
:1019E00009F063C0411161C08091E80082FDC9CF58
:1019F0008091F101882329F2853019F28091E80065
:101A000083FFF2CFBECF4132510509F43FC04232CD
:101A1000510509F001CF8330910508F0FDCEFC019E
:101A2000EE0FFF1FE45EFE4F0190F081E02D875E18
:101A30009E4FDC018C9190E01DC082E190E0E8E2D5
:101A4000F2E0BECF332721303105C1F060F0223003
:101A5000310509F0E1CEEAE3F2E0E4918E2F90E067
:101A6000EAE3F2E007C0E6E8F2E0E4918E2F90E0CE
:101A7000E6E8F2E0009709F4CFCEA2CFE6E7F2E085
:101A8000E4918E2F90E0E6E7F2E0F4CF8330910509
:101A900008F0C2CE880F991FFC01EE5DFE4F019049
:101AA000F081E02D89E090E08BCF8091F1018823D7
:101AB00009F467CF853009F464CF8091E80083FD95
:101AC00060CF8091E80082FD8FCF8091E80080FF99
:101AD00085CF8091F20090E02115310519F0883012
:101AE000910550F041E0089709F040E08091E8004E
:101AF0008E778093E80072CF44914093F100319645
:101B0000215031090196E8CF803809F085CE8091C7
:101B1000E800877F8093E8008091E8018093F100DE
:101B200070CE811179CE0091EB01023008F074CEB5
:101B30008091E800877F8093E8000093E8010E948D
:101B40006D0A002399F084E08093F10142E061EC9A
:101B500081E00E948C0A42E061EC82E00E948C0AE3
:101B600046E261EC83E00E948C0A56CE8091E3004D
:101B700087FDE9CF81E0E8CFEF92FF920F931F93AB
:101B8000CF937C018B010E943E0AC82F811119C09E
:101B90008091E80085FD0DC08091E8008E778093EC
:101BA000E8000E94BE0A0E943E0A882389F3C82FDB
:101BB00008C0F70181917F018093F1000150110964
:101BC00039F78C2FCF911F910F91FF90EF900895CF
:101BD0008091DD0108958091C601811113C09FB7E6
:101BE000F8944091D2025091D3026091D402709146
:101BF000D5029FBF443C59406105710518F081E052
:101C00008093C6010895EF92FF920F931F93CF9395
:101C1000DF93D82F0FB607FE46C08091F1018430C4
:101C200079F08091030190E001962091050130E068
:101C300082239323209104012817190609F0C9C0B3
:101C40000E94EB0D81110FC08091030190E001967D
:101C50002091050130E0822393232091040128176D
:101C6000190609F0B6C00E9451088C01C091E90024
:101C7000CF708091EC0080FD37C080E0C82B83E0FE
:101C80008093E90085E0E82E8091EB0085FD08C097
:101C90008091EB0080FF04C08091EE0087FD44C07E
:101CA000CF70C093E900E09103018E2F90E0019680
:101CB0002091050130E0822393232091040128170D
:101CC000190609F47EC08091010190910201E80F8C
:101CD000F92FF11DD083809103018F5F9091050151
:101CE0008923809303016DC080E8C8CFE091010192
:101CF000F0910201E80FF11D90818F5F20910501A5
:101D00008223809304019093F1008091E80085FD87
:101D10000BC08091E80080FF07C08091E8008E77BB
:101D20008093E800E092000180910401909103010A
:101D3000981741F19091E80095FDD8CF80E029C037
:101D40001092F1002EC08091030190E00196209145
:101D5000050130E0822393232091040128171906FE
:101D600009F09ECFF0900001FF2009F499CF0E9466
:101D700051088017910709F487CFFA94F092000177
:101D80008C0182CF8091E80085FFD8CFD093F100FD
:101D900081E09091F200992379F09091E80090FF12
:101DA0000BC09091E80095FDCBCF9091E8009E7715
:101DB0009093E800E0920001882329F2CF70C0934D
:101DC000E90080E0DF91CF911F910F91FF90EF909C
:101DD0000895E091030177CF8330C9F128F4813071
:101DE00061F0823019F10895853009F452C008F489
:101DF0003FC0863009F45EC00895809117016817CE
:101E000090F4861B80931701809117011F928F9386
:101E100082E799E09F938F930E9457060F900F904F
:101E20000F900F90089510921701EECF8091160138
:101E3000681750F4861B80931601809116011F923B
:101E40008F9380E699E0E6CF10921601F6CF80914D
:101E50001501681750F4861B8093150180911501B8
:101E60001F928F938DE499E0D5CF10921501F6CF94
:101E700080911401681750F4861B8093140180919F
:101E800014011F928F9388E399E0C4CF109214013C
:101E9000F6CF80911301681750F4861B80931301CD
:101EA000809113011F928F938FE199E0B3CF10922D
:101EB0001301F6CF80911201681750F4861B8093AE
:101EC0001201809112011F928F9384E099E0A2CFBA
:101ED00010921201F6CF833009F445C028F4813006
:101EE00061F0823049F10895853009F46AC008F440
:101EF00051C0863009F47CC0089580911701482FA5
:101F0000460F5527551F4F3F510594F4680F6093B6
:101F10001701809117011F928F9385EF98E09F938F
:101F20008F930E9457060F900F900F900F90089577
:101F30008FEF80931701EDCF80911601482F460F48
:101F40005527551F4F3F510554F4680F60931601F4
:101F5000809116011F928F9383EE98E0E0CF8FEF70
:101F600080931601F5CF80911501482F460F552714
:101F7000551F4F3F510554F4680F60931501809130
:101F800015011F928F9380ED98E0C9CF8FEF80935A
:101F90001501F5CF80911401482F460F5527551F85
:101FA0004F3F510554F4680F609314018091140160
:101FB0001F928F938BEB98E0B2CF8FEF8093140139
:101FC000F5CF80911301482F460F5527551F4F3FDE
:101FD000510554F4680F60931301809113011F920F
:101FE0008F9382EA98E09BCF8FEF80931301F5CF18
:101FF00080911201482F460F5527551F4F3F51051D
:1020000054F4680F60931201809112011F928F9314
:1020100087E898E084CF8FEF80931201F5CFCF93BC
:10202000DF932091F4013091F5012817390701F170
:102030009093F5018093F401E091C902F091CA02F6
:102040003097B1F0EC010084F185E02D0995809185
:10205000D8028570853061F4DF93CF9388E992E0F0
:102060009F938F930E9457060F900F900F900F90A1
:10207000DF91CF910895CF93DF932091F2013091BA
:10208000F3012817390701F19093F3018093F201CE
:10209000E091C902F091CA023097B1F0EC010680DC
:1020A000F781E02D09958091D8028570853061F423
:1020B000DF93CF938AE892E09F938F930E94570615
:1020C0000F900F900F900F90DF91CF9108958FECAC
:1020D00099E00E94BE051F9281E08F931F9285E0D8
:1020E0008F9381E899E09F938F930E9457060F90FA
:1020F0000F900F900F900F900F900895CF938091B5
:10210000D80283FF7EC084E294E00E94BE058091E5
:10211000CD021F928F938FE194E09F938F930E9443
:1021200057068DE194E00E94BE058091CE02282FD3
:10213000082E000C330B3F938F938AE194E09F931A
:102140008F930E94570688E194E00E94BE0580911B
:10215000CF02282F082E000C330B3F938F9385E17D
:1021600094E09F938F930E94570683E194E00E942E
:10217000BE058091D002282F082E000C330B3F9310
:102180008F9380E194E09F938F930E9457068EE097
:1021900094E00E94BE058091D102282F082E000CE9
:1021A000330B3F938F938BE094E09F938F930E9428
:1021B000570688E094E00E94BE058091C8021F92F5
:1021C0008F9385E094E09F938F930E94570683E05E
:1021D00094E00E94BE058091C7021F928F9380E019
:1021E00094E09F938F930E9457068DEF93E00E9497
:1021F000BE058DB79EB74C960FB6F8949EBF0FBE26
:102200008DBFE091C902F091CA023097F1F1C091FF
:10221000CD020480F581E02D8DEC92E00995C0930C
:10222000CD028091D80283FF30C08091D102282F47
:10223000082E000C330B3F938F938091D002282FF0
:10224000082E000C330B3F938F938091CF02282FE1
:10225000082E000C330B3F938F938091CE02282FD2
:10226000082E000C330B3F938F931F92CF9387E47C
:1022700094E09F938F930E9457068DB79EB70C965C
:102280000FB6F8949EBF0FBE8DBF0E945108909369
:10229000CC028093CB02CF9108950F931F93CF93DD
:1022A000DF938091B5029091B402892B8093B401A1
:1022B0009091B302992389F0892B8093B401E5EBC7
:1022C000F1E02CEB31E080E0919191118F5F2E17BE
:1022D0003F07D1F781111092B302E091C902F0914A
:1022E000CA023097B1F10280F381E02D84EB91E0D6
:1022F00009958091D80282FF2CC080FF04C082E73C
:1023000093E00E94BE05D0E0C0E00CE613E08091AF
:10231000D80280FF0EC0FE01EC54FE4F80811F9258
:102320008F931F930F930E9457060F900F900F905B
:102330000F902196C830D10551F78091D80280FFC7
:1023400008C08AE693E0DF91CF911F910F910C9422
:10235000BE05DF91CF911F910F9108951092B502A4
:102360001092B402E4EBF1E0118212821382148223
:102370001582168217820E944D1185E0EDECF2E085
:10238000DF011D928A95E9F71092C8021092C702E8
:102390000E947E1090E080E00E943B1090E080E080
:1023A0000C940F10CF93C82F1F928F938AEC9AE052
:1023B0009F938F930E94570681E090E0A0E0B0E0E9
:1023C00004C0880F991FAA1FBB1FCA95D2F780931C
:1023D000D9029093DA02A093DB02B093DC020F9053
:1023E0000F900F900F90CF910C94AE11882341F075
:1023F00080959091B50289238093B5020C944D117C
:102400000895882339F09091B502892B8093B50205
:102410000C944D1108958823E1F19CEF980F913AA7
:1024200068F4E4EBF1E09281891301C012823196E5
:1024300041E0EA3BF407B9F70C944D1190E2980F94
:10244000983088F4877021E030E0A90102C0440F81
:10245000551F8A95E2F7CA0180959091B5028923AC
:102460008093B502E9CF9BE5980F933020F490E07C
:1024700080E00C943B1098E5980F973120F490E0A1
:1024800080E00C940F10803F20F00E9460060C94B6
:102490007E100895CF938091C4019091C501981347
:1024A00004C0C0E08C2FCF91089590E0FC01E4546B
:1024B000FE4FC0810196877099278093C401CC2379
:1024C00081F31F92CF9387E591E09F938F930E94B2
:1024D000570685E591E00E94BE05EC2FE695E6954E
:1024E000E6959C2F977021E030E0A90102C0440FCF
:1024F000551F9A95E2F7CA010F900F900F900F9019
:10250000C7FF0FC0EF70F0E0E954FD4F4081242F6A
:1025100030E02823392380958423232B19F28083EC
:10252000C1CFF0E0E954FD4F2081422F50E0482315
:102530005923452B09F0B6CF822BF1CFCF93DF93F0
:1025400000D01F92CDB7DEB72091F101243041F5C4
:1025500020911001222321F123E029839B838A8388
:1025600082E08093E9008FEF9091E800815095FD23
:1025700006C095ED9A95F1F700008111F5CF809195
:10258000E80085FF0DC050E040E063E070E0CE0160
:1025900001960E94BC0D8091E8008E778093E80040
:1025A0000F900F900F90DF91CF910895CF93DF930D
:1025B00000D01F92CDB7DEB72091F101243081F514
:1025C00020911001222361F119821A821B8222E0DC
:1025D00029838138910520F0805891099B838A8353
:1025E00082E08093E9008FEF9091E800815095FDA3
:1025F00006C095ED9A95F1F700008111F5CF809115
:10260000E80085FF0DC050E040E063E070E0CE01DF
:1026100001960E94BC0D8091E8008E778093E800BF
:102620000F900F900F90DF91CF9108952091F101BD
:10263000243049F522E02093E9002FEF3091E800A3
:10264000215035FD06C035ED3A95F1F70000211116
:10265000F5CF2091E80025FF16C02091100150E031
:1026600040E063E070E0222339F021E02093F100A4
:1026700050E040E065E070E00E94BC0D8091E80011
:102680008E778093E8000895CF93DF932091F10136
:10269000243011F521E02093E90021E8215021F0B8
:1026A0003091E80035FF1BC02091E80025FF14C0E1
:1026B000EC0150E040E068E070E00E94BC0D8091C9
:1026C000E8008E778093E80088E0FE01AEEDB1E08F
:1026D00001900D928A95E1F7DF91CF910895EFE394
:1026E000F1E03197F1F700C00000D8CFCF938732E7
:1026F00008F043C08E3108F036C28E3009F4C9C1EB
:10270000B8F4873009F4ABC148F4863009F494C1B9
:1027100089E696E00E94BE0580E09FC1883009F4FA
:1027200055C08B30A9F785EA95E00E94BE0582C1AD
:10273000863109F4D8C178F4803151F79091D802EC
:10274000892F877F93FF88608093D80283FFB1C170
:1027500088E098E095C1893109F4AEC18B31C1F6AA
:102760009091D802892F8D7F91FF82608093D8024B
:1027700081FF8CC181E498E083C18833A1F250F4D9
:10278000893221F0853311F0873211F680E00E9402
:10279000D21150C18334D1F328F48A3308F4B8CF6E
:1027A0008953F5CF883409F0B3CF0E94AE1187E684
:1027B00098E00E94BE059FEF23ED80E391502040FA
:1027C0008040E1F700C000000E94C3098CE798E058
:1027D0000E94BE0585E995E00E94BE0583E090E079
:1027E0000E9493221F928F9382E995E09F938F938B
:1027F0000E94570680E995E00E94BE0582E090E0C5
:102800000E949322C82F8DE795E00E94BE051F927B
:10281000CF9388E795E09F938F930E94570686E7B2
:1028200095E00E94BE058CE695E00E94BE058C2FC7
:1028300081701F928F9389E695E09F938F930E94FA
:10284000570687E695E00E94BE058DE595E00E945B
:10285000BE05C1FB882780F91F928F938AE595E01A
:102860009F938F930E94570688E595E00E94BE05CE
:102870008CE495E00E94BE05C2FB882780F91F9278
:102880008F9389E495E09F938F930E94570687E486
:1028900095E00E94BE058EE395E00E94BE05C3FB55
:1028A000CC27C0F91F92CF938BE395E09F938F9332
:1028B0000E94570689E395E00E94BE0584E090E0FF
:1028C0000E949322C82F85E295E00E94BE051F92C8
:1028D000CF9380E295E09F938F930E9457068EE1FD
:1028E00095E00E94BE0585E095E00E94BE058C2F14
:1028F00081701F928F9382E095E09F938F930E9447
:1029000057068DB79EB780960FB6F8949EBF0FBE40
:102910008DBF80E095E00E94BE0589EE94E00E94A4
:10292000BE05C1FB882780F91F928F9386EE94E045
:102930009F938F930E94570684EE94E00E94BE05F9
:1029400082ED94E00E94BE05C2FB882780F91F92A9
:102950008F938FEC94E09F938F930E9457068DEC9A
:1029600094E00E94BE058BEB94E00E94BE05C3FB81
:10297000882780F91F928F9388EB94E09F938F9321
:102980000E94570686EB94E00E94BE058CEA94E014
:102990000E94BE05C4FB882780F91F928F9389EAA5
:1029A00094E09F938F930E94570687EA94E00E94D9
:1029B000BE0585E994E00E94BE05C5FB882780F925
:1029C0001F928F9382E994E09F938F930E94570602
:1029D00080E994E00E94BE0584E794E00E94BE0571
:1029E000C6FB882780F91F928F9381E794E09F931D
:1029F0008F930E9457068FE694E00E94BE0587E6FB
:102A000094E00E94BE05C7FBCC27C0F91F92CF936C
:102A100084E694E09F938F930E94570682E694E0A9
:102A20000E94BE058DB79EB74C960FB6F8949EBF18
:102A30000FBE8DBF81E011C08091D802817F8E7F53
:102A40008093D80282E496E00E94BE0588E798E071
:102A50000E94BE0581E08093D702CF9108958091B6
:102A6000D80280FF0BC08AE598E00E94BE058091E5
:102A7000D802817F8E7F8093D802DCCF8EE498E0ED
:102A80000E94BE058091D8028160F5CF83E398E073
:102A90004CCE9091D802892F8B7F92FF84608093D7
:102AA000D80282FF03C084E298E0EACF84E198E094
:102AB0003CCE8BEF97E039CE8CEE97E00E94BE05BE
:102AC00080EC97E00E94BE0585E797E00E94BE0576
:102AD0008FE497E00E94BE0580E097E00E94BE056B
:102AE00084ED96E022CE86EC96E00E94BE050E9420
:102AF000A0091F928F938CEA96E09F938F930E9478
:102B00005706809111011F928F9385E996E09F935C
:102B10008F930E9457068091D6021F928F9382E86E
:102B200096E09F938F930E9457062FB7F894809159
:102B3000D2029091D302A091D402B091D5022FBFBE
:102B4000BF93AF939F938F938BE696E09F938F9362
:102B50000E9457068DB79EB742960FB6F8949EBF57
:102B60000FBE8DBF67CF8D5112CECF93882309F44E
:102B7000ABC0C82F8CEF8C0F813A08F051C1809107
:102B8000D702813059F1F8F0823009F455C0109223
:102B9000D702A6EBB1E0EFEF80E09D91C91781F07D
:102BA000EF3F19F4911101C0E82F8F5F8630A9F72C
:102BB000EF3F31F00E2E000CFF0BEC54FE4FC283A2
:102BC000CF910C944D118091B4018152823008F75D
:102BD0008C2F0E947613811177C0DBCF8091B401D6
:102BE00081528230A8F3C431C9F048F4CB3059F097
:102BF000C031C1F088EA92E00E94BE0511C0C9321E
:102C000069F0C833B9F782E496E00E94BE058EEA07
:102C100092E00E94BE0581E08170DDCF1092D70264
:102C200080E0FACF0E9467108AEA92E00E94BE0517
:102C300082E08093D702EFCFC432C8F4CE3108F0DF
:102C4000BEC0CB30E1F040F4C73009F4CFC087E517
:102C500093E0CF910C94BE05C331C1F1C431B9F7F3
:102C60008091F601882349F11092F6010AC0CB3415
:102C700009F4BAC0C0F4C93299F3C83341F70E94CD
:102C800067108091F601882309F4C7C01F928F93C3
:102C900081E593E09F938F930E9457060F900F90CA
:102CA0000F900F9011C0C13509F498C0C23509F4D6
:102CB0008FC0CE3461F66AE092C086E693E00E944F
:102CC000BE0581E08093D702CF91089580E493E020
:102CD0000E94BE058EE293E00E94BE05809117011E
:102CE0001F928F938BE293E09F938F930E945706DE
:102CF00089E293E00E94BE0587E193E00E94BE0551
:102D0000809116011F928F9384E193E09F938F939C
:102D10000E94570682E193E00E94BE0583E093E0A3
:102D20000E94BE05809115011F928F9380E093E071
:102D30009F938F930E9457068EEF92E00E94BE05EC
:102D40008DEE92E00E94BE05809114011F928F9338
:102D50008AEE92E09F938F930E94570688EE92E04E
:102D60000E94BE0583ED92E00E94BE058091130192
:102D70001F928F9380ED92E09F938F930E9457064E
:102D80008EEC92E00E94BE0587EB92E00E94BE05A9
:102D9000809112011F928F9384EB92E09F938F9307
:102DA0000E94570682EB92E00E94BE058DB79EB747
:102DB00048960FB6F8949EBF0FBE8DBF62CFCE511E
:102DC000EC2FF0E0E85DFE4F80818093F60159CF53
:102DD00061E08091F6010E946B0F53CF61E080911A
:102DE000F6010E94EC0E4DCF6AE0F3CF8EE18093A6
:102DF000170182E3809316018AE08093150184E134
:102E00008093140188E08093130188E2809312017B
:102E100089E593E00E94BE0534CF8EE493E019CF9C
:102E200080E28C0F883068F4C77021E030E001C088
:102E3000220FCA95EAF78091B502822B8093B502E2
:102E4000BFCE8BE58C0F833068F481E890E0C53A03
:102E500031F083E890E0C63A11F482E890E0CF9137
:102E60000C943B1088E58C0F873108F068C082EE27
:102E700090E0C83A09F460C089EE90E0C93A09F4DC
:102E80005BC08AEE90E0CA3A09F456C085EB90E048
:102E9000CB3A09F451C086EB90E0CC3A09F44CC02F
:102EA00083EB90E0CD3A09F447C084EB90E0CE3A52
:102EB00009F442C087EB90E0CF3AF1F18CEC90E05E
:102EC000C13BD1F18DEC90E0C03BB1F183E891E0E2
:102ED000C23B91F18AE891E0C33B71F182E991E054
:102EE000C43B51F184E991E0C53B31F181E292E0CC
:102EF000C63B11F183E292E0C73BF1F084E292E03D
:102F0000C83BD1F085E292E0C93BB1F086E292E0A5
:102F1000CA3B91F087E292E0CB3B71F08AE292E00B
:102F2000CC3B51F08FE690E0CD3B31F090E080E07B
:102F3000CE3B11F480E790E0CF910C940F10CF3B83
:102F400069F40E94AE119FEF20E782E0915020408B
:102F50008040E1F700C000000E94C309C03F08F4B0
:102F6000B3CE8C2F0E946B07CF910C947E10CF9222
:102F7000DF92EF92FF920F931F93CF93DF9300D0D6
:102F800000D01F92CDB7DEB76C0185E0F601DE01FF
:102F9000119601900D928A95E1F7F60140815181D9
:102FA0002381348191E02115310531F05F3F19F41F
:102FB00091E04F3F09F090E090FD99C0F601028149
:102FC000F580F2949FE0F92249835A830B83722F94
:102FD0003D832C83602F8D810E945D08182FE92F7F
:102FE000E295EF70EF3008F082C0F0E0E650F84E66
:102FF0000C9422240918091847184718BD18EF180F
:103000007718771805197718DB19DB1977187718EF
:10301000971AF92FFF70FF2E907F19F0F29480EF2E
:10302000F8220023C9F0FF2039F08091B402F82A79
:10303000F092B4020E944D11812F0F900F900F90CB
:103040000F900F90DF91CF911F910F91FF90EF9014
:10305000DF90CF900C94B515812F0E940B12FF20AA
:1030600009F445C0F0948091B402F822F092B402C1
:103070000F900F900F900F900F90DF91CF911F91B5
:103080000F91FF90EF90DF90CF900C944D11892F0E
:103090008F70907F903211F08295807F112379F0AC
:1030A000113009F449C0002309F455C0FF2059F03C
:1030B000F601958190FF8DC19F70958304C0002318
:1030C00021F1F1100FC00F900F900F900F900F9003
:1030D000DF91CF911F910F91FF90EF90DF90CF90F4
:1030E0000C94011221E0F212EECF8093B3020F9004
:1030F0000F900F900F900F90DF91CF911F910F9134
:10310000FF90EF90DF90CF900895F11011C01092D2
:10311000B3020F900F900F900F900F90DF91CF910F
:103120001F910F91FF90EF90DF90CF900C94F611CC
:1031300091E0F912ECCFDBCF002349F0E5E0EF1589
:10314000B0F29091B502982309F4BDCFE2CFF4E03C
:10315000FF1568F2DECFFF20E1F2812F0F900F9074
:103160000F900F900F90DF91CF911F910F91FF90D3
:10317000EF90DF90CF900C940B12892F8695869557
:103180008370C1F0813009F0B2CF812F93700111AB
:1031900002C090E080E00F900F900F900F900F9082
:1031A000DF91CF911F910F91FF90EF90DF90CF9023
:1031B0000C940F10812F9370011102C090E080E0F9
:1031C0000F900F900F900F900F90DF91CF911F9164
:1031D0000F91FF90EF90DF90CF900C943B10002365
:1031E00089F00E946B070F900F900F900F900F9037
:1031F000DF91CF911F910F91FF90EF90DF90CF90D3
:103200000C947E100E946006EECF892F837009F027
:1032100064C001116CCF812F829586958770880FCD
:10322000880F412F4F70C42ED12CF12CE12C082E89
:1032300004C0CC0CDD1CEE1CFF1C0A94D2F740E04D
:1032400050E0BA0114FF11C00FE010E020E030E0C0
:1032500004C0000F111F221F331F8A95D2F7B90136
:10326000A80140955095609570950091D9021091F4
:10327000DA022091DB023091DC02969596959370EC
:103280009230E9F028F5913089F04C295D296E29BA
:103290007F2940235123622373234093D902509303
:1032A000DA026093DB027093DC0221CFC02AD12ABC
:1032B000E22AF32A4C295D296E297F29EECF4C2979
:1032C0005D296E297F294027512762277327E5CF83
:1032D0004023512362237323EDCF8695002311F001
:1032E000892F8170882309F402CF812F82958695DA
:1032F0008770880F880F412F4F70C42ED12CF12C6E
:10330000E12C082E04C0CC0CDD1CEE1CFF1C0A9422
:10331000D2F740E050E0BA0114FF11C00FE010E016
:1033200020E030E004C0000F111F221F331F8A95D8
:10333000D2F7B901A801409550956095709500911C
:103340002F02109130022091310230913202969575
:10335000969593709230E9F028F5913089F04C29D8
:103360005D296E297F2940235123622373234093D3
:103370002F02509330026093310270933202B7CE25
:103380000C291D292E293F29402B512B622B732BF1
:10339000EECF4C295D296E297F29402751276227CE
:1033A0007327E5CF40235123622373234C295D29E2
:1033B0006E297F29DCCF803F09F44EC0D0F480E431
:1033C000810F803270F1002309F4ACC0FF2009F4B2
:1033D000A6C0812F0E94B515193309F099C0FFEFDF
:1033E00021EE84E0F15020408040E1F700C0000071
:1033F0007ECE823F09F470C008F45BC0833F19F7AA
:10340000002309F47CC0292F2F7181E090E0A0E017
:10341000B0E004C0880F991FAA1FBB1F2A95D2F7DE
:103420003AC0E12FE071FE2E892F8F71002351F0F9
:103430000E942A09812F8295807FF11044CE812F2E
:103440008F7041CE0E940609812F8295807FF110F6
:1034500060CE812F8F705DCE002331F1F4E0FF1537
:1034600008F445CE292F2F7181E090E0A0E0B0E074
:1034700004C0880F991FAA1FBB1F2A95D2F740913D
:103480002F025091300260913102709132028427F4
:103490009527A627B72780932F0290933002A093F9
:1034A0003102B093320223CE25E02F1508F41FCE4F
:1034B000D9CF892F8F71002399F00F900F900F9023
:1034C0000F900F90DF91CF911F910F91FF90EF9090
:1034D000DF90CF900C942A09892F8F71002369F314
:1034E0000F900F900F900F900F90DF91CF911F9141
:1034F0000F91FF90EF90DF90CF900C9406091092FF
:103500002F02109230021092310210923202EFCD4F
:10351000133509F464CF173409F0E9CD60CF892F52
:103520008F71CBCFF11019CE892F8F71D9CF811127
:10353000DECD002309F4DBCD0E94AE118FEF90E7C2
:10354000E2E081509040E040E1F700C000000E94BE
:10355000C3091F93CF93DF938091FC01807FB1F467
:103560008091F901882391F020912E021091FD01A4
:10357000C091F701D091F801A091FA01B091FB013F
:1035800041E0CF3F09F040E0121304C0DF91CF913A
:103590001F91089581E0109721F0842FDF3F09F0FB
:1035A00080E030E080FD33C0C90166E070E00E9439
:1035B000FD23FC01E250FE4F81818D1328C08081E4
:1035C0008C1325C08281811122C0838194818A1B42
:1035D0009B0B883C9105D8F48091FC018F70806131
:1035E0008093FC01C90166E070E00E94FD23FC01AC
:1035F000ED5FFD4F90819F709061908387EF91E028
:103600000E94B717DF91CF911F910C944A092F5F49
:103610003F4F2770B9CF9F92AF92BF92CF92DF9268
:10362000EF92FF920F931F93CF93DF93CDB7DEB747
:1036300061970FB6F894DEBF0FBECDBF8C0185E059
:10364000F801DE011D9601900D928A95E1F7F801CF
:1036500040812181F280C380D4809091F701309124
:10366000F8016091FA017091FB0181E0611571052B
:1036700031F03F3F19F481E09F3F09F080E0F82FDF
:10368000F1709F2E80FD4EC187EFA82E81E0B82EED
:10369000E090F901F601E61BF70BEE2009F404C1F6
:1036A0008091FC01582F507FE83CF10508F0BDC027
:1036B000511183C0EF2C321322C0941320C0F1109B
:1036C0001EC08F7080618093FC01C5010E94B717F6
:1036D0008091FC01F80185838E2D61960FB6F894D8
:1036E000DEBF0FBECDBFDF91CF911F910F91FF9035
:1036F000EF90DF90CF90BF90AF909F90089581E0C2
:10370000C114D10431F02F3F19F481E04F3F09F08B
:1037100080E080FD14C081E08F25F82FF170BF2E6E
:10372000E0912E023091FD0180FD22C0FF20A1F228
:103730008091FC0181608093FC01E12CCDCF80E081
:10374000ECCFF0E0CF0166E070E00E94FD23DC01E9
:10375000A250BE4F11968C911197281307C08C91DF
:10376000481304C012968C918F11E0CF3196E77008
:10377000E313E7CF7C2DD98AC88A522F6F2D898910
:103780000E945D08292F22952F70223050F024309E
:1037900078F49F7051F0F8019581907F31F4E92C15
:1037A0009BCF9F7011F08823D1F3805E8830B8F3EF
:1037B000C8010E94B7179B2CF2CF321306C0941396
:1037C00004C0F801FF2009F48AC04D872E87FF86C8
:1037D0007C2DD98AC88A522F6F2D89890E9454095D
:1037E000882309F4AEC0FF2009F4ABC08091FC012E
:1037F000803270F02091F7013091F80138872F83E3
:103800001986DB86CA868C87CE0107960E94B71779
:1038100086E0F801A7EFB1E001900D928A95E1F7FB
:103820000E94A91AEE24E39457CF51110AC087EFE2
:1038300091E00E94B71786E0F50111928A95E9F7A9
:103840007CCF32130FC094130DC0F1100BC0F801E0
:103850008583C8010E94B71786E0F50111928A9509
:10386000E9F73ACF4D872E87FF867C2DD98AC88A03
:10387000522F6F2D89890E945409882309F461C051
:10388000FF2009F45EC08091FC01803208F2209193
:10389000F7013091F8013A8329831B82DD82CC82C3
:1038A0008E83CE010196B2CFE83CF105A8F6EF2C4D
:1038B000FF2009F446C032131FC094131DC080912D
:1038C000FC0180FD10C0982F907F69F0F80185837E
:1038D000903F31F0982F907F905F8F70892B858378
:1038E000C8010E94B71786E0F801A7EFB1E0019088
:1038F0000D928A95E1F7F0CE4D872E87FF867C2DBD
:10390000D98AC88A522F6F2D89890E945409811142
:103910007FCF8091FC0181608093FC01C8010E94EF
:10392000B717DACEFF2069F04D872E87FF867C2DF2
:10393000D98AC88A522F6F2D89890E945409811112
:1039400067CFC8010E94B7176DCFCF93DF93CDB774
:10395000DEB767970FB6F894DEBF0FBECDBF4B8BB7
:103960005C8B6D8B7E8B8F8B1A8A198A85E0FE01AA
:103970007396DE011D9601900D928A95E1F786E01F
:10398000FE013D96DE01179601900D928A95E1F7B2
:10399000CE0107960E940B1B811138C086E0FE0104
:1039A0003796DE01119601900D928A95E1F79F817D
:1039B00088852A853B85232B39F08F3F19F481E0D8
:1039C0009F3F19F080E001C081E080FD1FC0809121
:1039D000FD0190E09C012F5F3F4F277033274091FE
:1039E0002E024217130661F166E070E00E94FD238B
:1039F000DC01A250BE4F96E0FE01319601900D927F
:103A00009A95E1F72093FD010E944A0980912E02C8
:103A10009091FD01891709F190E066E070E00E9445
:103A2000FD2382509E4F0E940B1B8823B1F0809192
:103A30002E0290E001968770992780932E02E6CFA0
:103A40000E94AE111092FD0110922E0286E0E7EF67
:103A5000F1E0DF011D928A95E9F767960FB6F894B9
:103A6000DEBF0FBECDBFDF91CF9108956DEE7EEF2B
:103A700090E080E00E94AF2260E082E090E00E944F
:103A8000A12260E083E090E00E94A12260E084E057
:103A900090E00E94A12260E085E090E00C94A122D9
:103AA00078941F920F920FB60F9211248F939F93C9
:103AB000AF93BF938091D2029091D302A091D40290
:103AC000B091D5020196A11DB11D8093D2029093B1
:103AD000D302A093D402B093D502BF91AF919F912E
:103AE0008F910F900FBE0F901F9018951F920F92FD
:103AF0000FB60F9211248F939F93AF93BF93809132
:103B0000B602811113C08091D2029091D302A0918C
:103B1000D402B091D5024196A11DB11D8093D2026D
:103B20009093D302A093D402B093D502BF91AF91EA
:103B30009F918F910F900FBE0F901F9018951F921D
:103B40000F920FB60F9211242F933F934F935F93D1
:103B50006F937F938F939F93AF93BF93EF93FF9355
:103B60008091E10082FF09C08091E20082FF05C0E0
:103B70008091E1008B7F8093E1008091E10080FFE4
:103B80001FC08091E20080FF1BC08091E2008E7F09
:103B90008093E2008091E20080618093E200809156
:103BA000D80080628093D80019BC85E08093F10131
:103BB0008091DD018093DC011092DD010E94AE1145
:103BC0008091E10084FF2DC08091E20084FF29C034
:103BD00084E089BD86E089BD09B400FEFDCF8091F7
:103BE000D8008F7D8093D8008091E1008F7E8093F4
:103BF000E1008091E2008F7E8093E2008091E200FC
:103C000081608093E2008091E801882309F45EC01E
:103C100084E08093F1010E94AE118091DC018093D9
:103C2000DD018091E10083FF40C08091E20083FFCD
:103C30003CC08091E100877F8093E10082E0809327
:103C4000F1011092E8018091E1008E7F8093E10004
:103C50008091E2008E7F8093E2008091E20080619B
:103C60008093E20042E060E080E00E948C0A81E004
:103C7000809311011092D6021092DD0198E0EEEDD2
:103C8000F1E0DF011D929A95E9F71092B5011092CB
:103C9000B6011092B7011092B8011092B9011092BA
:103CA000BA011092BB0180931001FF91EF91BF9177
:103CB000AF919F918F917F916F915F914F913F91C4
:103CC0002F910F900FBE0F901F9018958091E300D9
:103CD00087FD02C081E09DCF83E09BCFCF93DF9330
:103CE000CDB7DEB72C970FB6F894DEBF0FBECDBFB1
:103CF00084B7877F84BF0FB6F894A8958091600041
:103D0000886180936000109260000FBE80E890E0B0
:103D10000FB6F89480936100909361000FBE83E02A
:103D20009EE0909333018093320186E091E090937E
:103D3000CA028093C9028BEB91E00E94BE050E94EB
:103D4000AC09809163008E7F8093630081E0809353
:103D5000DB011092E2001092E1008091D8008F7791
:103D60008093D8008091D80080688093D80080919B
:103D7000D8008F7D8093D80084E089BD86E089BD1E
:103D800009B400FEFDCF1092F1011092E8011092EB
:103D9000E7011092E60142E060E080E00E948C0AB8
:103DA0008091E1008E7F8093E1008091E20081604C
:103DB0008093E2008091E20088608093E20080912D
:103DC000E0008E7F8093E000789482E084BD93E0F1
:103DD00095BD9AEF97BD80936E0087E68093CC00E7
:103DE0001092CD008091C90080698093C90087EC52
:103DF00092E0B7EBCB2EB2E0DB2EF60111926F0111
:103E00008E179F07D1F790E080E00E949B228D3EA5
:103E10009E4F11F00E94361D83E691E00E94BE0580
:103E200015E61150C9F48CE591E00E94BE0589E2C7
:103E300090E00E943F088111F7C08AE290E00E9462
:103E40003F0881110E94361D85E090E00E943F08E6
:103E5000882359F00E94C3090E944A128FE39CE90B
:103E60000197F1F700C00000DCCF82E090E00E94F3
:103E700093228093D80287E090E00E943F08882335
:103E800079F08BE190E00E943F08882309F4FAC1A1
:103E90009091D802892F8D7F91FF82608093D80204
:103EA0006091D80282E090E00E94A12284E090E03C
:103EB0000E9493228093C70180EE90E00E943F0809
:103EC000882341F09091C701892F8E7F90FF8160F8
:103ED0008093C70189E390E00E943F08882341F066
:103EE0009091C701892F8D7F91FF82608093C701D8
:103EF00082EE90E00E943F08882341F09091C70134
:103F0000892F8B7F92FF84608093C70186EE90E0BB
:103F10000E943F08882341F09091C701892F877F35
:103F200093FF88608093C70183EE90E00E943F0872
:103F3000882341F09091C701892F8F7E94FF806183
:103F40008093C70185E390E00E943F08882341F0F9
:103F50009091C701892F8F7D95FF80628093C70163
:103F600081E390E00E943F08882341F09091C701CF
:103F7000892F8F7B96FF80648093C70181E190E059
:103F80000E943F08882341F09091C701892F97FB39
:103F900087F980588093C7016091C70184E090E061
:103FA0000E94A12287E290E00E943F08182F8EE134
:103FB00090E00E943F08811112608FE190E00E9422
:103FC0003F088111146080E290E00E943F08811157
:103FD000186081E290E00E943F088111106182E246
:103FE00090E00E943F088111106283E290E00E94FD
:103FF0003F088111106484E290E00E943F0888230A
:1040000009F45FC11068612F83E090E00E94A12253
:10401000812F90E0B0E0A0E08093D9029093DA0283
:10402000A093DB02B093DC028091F101843009F0AF
:104030004FC10E94EB0D882309F44AC189EA91E03F
:104040000E94BE058BE991E00E94BE05F0E94F2E6B
:10405000F1E05F2EA8E16A2E712C8091F10185308C
:1040600009F439C10E944A1209EC11E0E7EBAE2EC7
:10407000E2E0BE2E312CF50121905F01F801908025
:10408000921409F468C08091D80281FF40C083E88F
:1040900091E00E94BE0527EB32E03C872B87F12C94
:1040A000E12CEB85FC852191FC87EB87229530E0A4
:1040B000C901880F991F880F991F8C7C359527950A
:1040C000359527952373822B90E028E131E03F93CB
:1040D0002F939C01220F331F2A7A9595879585751A
:1040E000822B1F928F93FF92EF9288E791E09F932C
:1040F0008F930E945706FFEFEF1AFF0A0FB6F8944E
:10410000DEBF0FBECDBF30E1E316F10451F6E12C66
:10411000FF24F3949224892D8F21C1F0EE823F82F7
:1041200091E08F2D822109F490E098870E94510838
:104130008160782F9A8789874E815F8168858A851B
:104140000E94A51CF80180818F258083E394FF0CD9
:10415000F8E0EF12E0CF33940F5F1F4F20E13212EF
:104160008ACF3FEF39833A831B820E9451088160D6
:10417000782F9D838C8349815A816B818D810E9428
:10418000A51C8091CB029091CC022FB7F89440915E
:10419000D2025091D3026091D4027091D5022FBF08
:1041A000FA01E81BF90B2091C8028091160190E0FA
:1041B000211107C08091170190E06AE070E00E9431
:1041C000FD23E817F90780F08091CE02F090CF022E
:1041D0001091D0020091D1028111B3C0F11073C1CE
:1041E000111171C101116FC10E94A0099091C80104
:1041F000891799F00E94A0098093C8019091D80274
:104200009570953051F41F928F935F924F920E9458
:1042100057060F900F900F900F902091E40030916F
:10422000E5008091D9019091DA012817390739F119
:104230008091E4009091E5009093DA018093D90198
:104240000E94EB0D8823D9F08091F1018430B9F4FC
:104250008091E9008F709091EC0090FFE0C090E8B1
:10426000892B93E09093E9009091EB0090FF04C0BC
:104270009091EE0097FDF1C08F708093E9000E944D
:10428000BE0AEBCE8EE090E00E943F08882339F012
:104290009091D802892F8B7F92FF8460FFCD80E1BF
:1042A00090E00E943F089091D802882329F0892F3E
:1042B000877F93FF8860F2CD892F8E7F90FF81608A
:1042C000EDCD1111A0CE83E090E00E949322A1CE0B
:1042D0000E94BE0AA9CE8091F101843011F11092A2
:1042E000B60280E40FB6F894A895609260000FBE05
:1042F0008093600083B7817F846083BF83B78160D0
:1043000083BF7894889583B78E7F83BF0FB6F89468
:10431000A895809160008861809360001092600091
:104320000FBE8091E701882309F497CE0E944A12BC
:10433000E7EBF2E081918111B0C0CE16DF06D1F734
:104340008CCE2F3F19F02F5F2093C802181624F44B
:104350000E941F078093CE028091CE0287FF05C086
:104360000E941F0781958093CE021F1424F40E949F
:104370001F078093CF028091CF0287FF05C00E9464
:104380001F0781958093CF026091CE02662331F1A1
:10439000F090CF02FF2011F1062E000C770B880B56
:1043A000990B0E94FC2223E333E343E35FE30E9483
:1043B00060230E94C4226093CE026F2DFF0C770B06
:1043C000880B990B0E94FC2223E333E343E35FE372
:1043D0000E9460230E94C4226093CF02111624F42D
:1043E0000E94E4068093D0028091D00287FF05C02E
:1043F0000E94E40681958093D002101624F40E9456
:10440000E4068093D1028091D10287FF05C00E940B
:10441000E40681958093D1020E947E10E5CE90E063
:104420001FCFE0910101F0910201E90FF11D208100
:104430009F5F309105019323909304012093F10035
:104440009091E80095FD09C09091E80090FF05C0AB
:104450009091E8009E779093E8009091040120915C
:104460000301291721F02091E80025FDDACF909172
:10447000F200992309F400CF9091E80090FFFCCE60
:104480009091E80095FD06C09091E8009E7790938A
:10449000E800F2CE1092F100F3CF84E089BD86E00F
:1044A00089BD09B400FEFDCF8091D8008F7D809337
:1044B000D8008091E00082608093E0008091E0006D
:1044C00081FDFCCFCACD2F3F09F03DCF4ECF1F92CB
:1044D0000F920FB60F9211242F933F934F938F9308
:1044E0009F93EF93FF938091C50190E09C012F5F14
:1044F0003F4F277033274091C401421741F030915C
:10450000CE0084549E4FFC0130832093C501FF915F
:10451000EF919F918F914F913F912F910F900FBEEF
:104520000F901F901895F999FECF92BD81BDF89A12
:10453000992780B50895A8E1B0E042E050E00C94DE
:10454000B622262FF999FECF1FBA92BD81BD20BD9C
:104550000FB6F894FA9AF99A0FBE019608950E9440
:10456000A122272F0C94A222DC01CB01FC01F99996
:10457000FECF06C0F2BDE1BDF89A319600B40D92AF
:1045800041505040B8F708950E94CB226894B11171
:104590000C945A2308950E943F2388F09F5798F067
:1045A000B92F9927B751B0F0E1F0660F771F881F38
:1045B000991F1AF0BA95C9F714C0B13091F00E9452
:1045C0005923B1E008950C945923672F782F882739
:1045D000B85F39F0B93FCCF3869577956795B39579
:1045E000D9F73EF490958095709561957F4F8F4FE8
:1045F0009F4F0895E89409C097FB3EF490958095ED
:10460000709561957F4F8F4F9F4F9923A9F0F92F98
:1046100096E9BB279395F695879577956795B79516
:10462000F111F8CFFAF4BB0F11F460FF1BC06F5FFC
:104630007F4F8F4F9F4F16C0882311F096E911C00E
:10464000772321F09EE8872F762F05C0662371F02F
:1046500096E8862F70E060E02AF09A95660F771F43
:10466000881FDAF7880F9695879597F9089557FD73
:104670009058440F551F59F05F3F71F04795880FD0
:1046800097FB991F61F09F3F79F087950895121667
:1046900013061406551FF2CF4695F1DF08C0161613
:1046A00017061806991FF1CF8695710561050894C4
:1046B0000895E894BB2766277727CB0197F90895DB
:1046C0000E9472230C94EC230E94DE2338F00E9497
:1046D000E52320F0952311F00C94D5230C94DB23D3
:1046E0000C945A230E94372378F39923C9F3552356
:1046F000B9F3950F50E0551FAA27EE27FF27BB27D8
:1047000000240894679520F4E20FF31FB41F0A1EDB
:10471000220F331F441FAA1F6695A9F7779530F41F
:10472000F30FB41F0A1E121E08F46395330F441FC3
:10473000AA1F221F769599F7879520F4B40F0A1EB9
:10474000121E631F440FAA1F221F331F8695A9F74D
:10475000862F712D602D11249F5750409AF0F1F053
:1047600088234AF0EE0FFF1FBB1F661F771F881FAD
:1047700091505040A9F79E3F510580F00C94D523ED
:104780000C945A235F3FE4F3983ED4F386957795D3
:104790006795B795F795E7959F5FC1F7FE2B880F53
:1047A000911D9695879597F9089597F99F6780E8E9
:1047B00070E060E008959FEF80EC089500240A9473
:1047C0001616170618060906089500240A941216EC
:1047D0001306140605060895092E0394000C11F41F
:1047E000882352F0BB0F40F4BF2B11F460FF04C0CC
:1047F0006F5F7F4F8F4F9F4F08950024552704C050
:10480000080E591F880F991F009729F07695679514
:10481000B8F37105B9F7802D952F089597FB072EF2
:1048200016F4009407D077FD09D00E94282407FCD5
:1048300005D03EF4909581959F4F089570956195B0
:104840007F4F0895EE0FFF1F0590F491E02D09941E
:10485000AA1BBB1B51E107C0AA1FBB1FA617B707A6
:1048600010F0A61BB70B881F991F5A95A9F78095C2
:0C4870009095BC01CD010895F894FFCF95
:10487C0005340100007FE80D44131613D6129E1266
:10488C0001012808140A321E00407F2215019600EF
:10489C007400E601FF011802010203040506070873
:0248AC00090001
:106800005300EA44E9448140040005000600070003
:10681000080009000A000B000C000D000E000F001C
:1068200010001100120013001400150016001700CC
:10683000180019001A001B001C001D001E001F007C
:10684000200021002200230024002500260027002C
:10685000280029002A002B002C002D002E002F00DC
:106860003000310035003300340035003600370089
:10687000380039003A003B003C003D003E003F003C
:1068800040004100420043004400450046004700EC
:10689000480049004A004B004C004D004E004F009C
:1068A000500051005200530054005500560057004C
:1068B000F1A159005A005B005C005D005E005F00C2
:1068C00060006100620063006400650036006700DC
:1068D000680069006A006B006C006D006E006F005C
:1068E00070007100720073003100E5008A008B00B7
:1068F000E000E100E200E300F1A1E500E600E700CE
:106900000100010001000100EA4401000100E2442D
:106910000100010001000100460001004A004B0097
:10692000010001004700480001000100E9440100A6
:106930000100010001000100010001003A003B00DC
:106940003C003D003E003F0040004100420043004B
:10695000010035004C0039000100440045005200A0
:1069600001000100010050004F0029004D004E00C1
:106970005100010044004500010001000100010038
:106980000100010044004500010001000100010078
:1069900001000100010001004900010001004D005B
:1069A0004A004E004B000100010001005400550058
:1069B00001000100010001000100010001000100CF
:1069C0000100010001000100010001006700010059
:1069D00001000100010001000100010001000100AF
:1069E0000100010001000100490001000100010057
:1069F000010001000100010001000100010001008F
:00000001FF
